:020000040000FA
:040000006A303A2800
:08000800A000030EA100831209
:100010008B1C32288B1031181428B11C3228643004
:10002000010203183128182800001628172818285C
:1000300019281A281B281C281D281E281F283110A3
:10004000B114A810031005190314AA0DA90DA80DC9
:10005000B00B322831152A08AF002908AE00280855
:10006000AD00B11081010B11210E8300A00E200EF6
:02007000090085
:0C007400203084008001840A6030040207
:10008000031C3C281230B0006A2283160C30850510
:1000900087018312850187010730990000309A009B
:1000A000103083168E008312603083168F00831207
:1000B0000030831691008312C830831681008312AA
:1000C00031309000003083168C00831210308B008A
:1000D000831600309B001C141A088312BC00851D77
:1000E00077233C1C8228831610309B001C141A08AE
:1000F0008312BD00831630309B001C141A08831233
:10010000C2000123831620309B001C141A0883129E
:10011000C1000130C1080319C10081018E018F01A6
:100120000B118B100B108C018B17A5203119BB20E4
:100130004722B30BA328031085190314B90DF0301F
:1001400039020319D62116239528640031180800B6
:100150000B1D08000B11B11031141230B000051D39
:10016000B628321483160113831208003210831646
:1001700001178312080031110130B7008B132030B2
:10018000370783169B001C141A088312A400A500CD
:10019000C030A5061030370783169B001C141A08C0
:1001A0008312A3000030370783169B001C141A0823
:1001B0008312A2008B17321CE32822090339A20004
:1001C000A309A409A50922082D02031DD02923088B
:1001D0002E02031DD02924082F02031D5D290130A2
:1001E0003702031DFA283C19F9283D18FA283D1456
:1001F0003E146B2202303702031D05293C190429E5
:10020000BD180529BD143E14722203303702031DA8
:1002100010293C190F293D1910293D153E1479224A
:1002200004303702031D1B293C191A29BD191B294B
:10023000BD153E14802205303702031D26293C19C6
:1002400025293D1A26293D163E14872206303702FD
:10025000031D31293C193029BD1A3129BD163E1420
:100260008E2207303702031D3C293C193B293D1BD8
:100270003C293D173E14952208303702031D4729BB
:100280003C194629BD1B4729BD173E149C22093045
:100290003702031D52293C19512942185229421490
:1002A0003E14A3220A303702031D5D293C195C2944
:1002B000C2185D29C2143E14AA2225082F02031D6C
:1002C000D02901303702031D6C293C196B293D1CD4
:1002D0006C293D103E14B12202303702031D7729EC
:1002E0003C197629BD1C7729BD103E14B522033078
:1002F0003702031D82293C1981293D1D82293D11A8
:100300003E14B92204303702031D8D293C198C2973
:10031000BD1D8D29BD113E14BD2205303702031DC0
:1003200098293C1997293D1E98293D123E14C12257
:1003300006303702031DA3293C19A229BD1EA3299B
:10034000BD123E14C52207303702031DAE293C19E9
:10035000AD293D1FAE293D133E14C9220830370296
:10036000031DB9293C19B829BD1FB929BD133E1475
:10037000CD2209303702031DC4293C19C329421C70
:10038000C42942103E14D1220A303702031DCF295E
:100390003C19CE29C21CCF29C2103E14D522D02927
:1003A000B70A0B30370203180800BE280130B60028
:1003B000B300B400B500B70085018701B113A520D3
:1003C000B30B162A031085190314B90DF030390246
:1003D00003193D2AB40B162A013037020319D9221A
:1003E000023037020319DD22033037020319E122FC
:1003F000043037020319E522053037020319E922D8
:10040000063037020319ED22073037020319F122B3
:10041000083037020319F522093037020319F9228F
:100420000A3037020319FD229630B400311DDF294E
:100430003111321C202A2D090339AD00AE09AF0954
:100440002F1CB1132F1CDF29B11BDF292E18DF2928
:10045000B1178B1320303707BB002F08BA00552285
:1004600010303707BB002E08BA005522003037077E
:10047000BB002D08BA0055228B1785018701B70AEA
:10048000B6010B303702031CDF29012308003E1C94
:1004900008003E101030BB003D08BA005522303035
:1004A000BB004208BA00552208008B133A08831695
:1004B0001C159A0083123B0883169B0055309D0043
:1004C000AA309D009C1464009C18632A1C1183129E
:1004D0008B1708000800051640084107D0000F08D8
:1004E000D1000800851640084107D2000F08D3004C
:1004F0000800051440084107D4000F08D500080083
:10050000851440084107D6000F08D700080087145B
:1005100040084107D8000F08D90008000715400817
:100520004107DA000F08DB00080007144008410704
:10053000DC000F08DD000800871640084107DE00D8
:100540000F08DF000800071640084107CC000F081D
:10055000CD000800871540084107CE000F08CF00E6
:10056000080005128E018F01080085128E018F018F
:10057000080005108E018F01080085108E018F0183
:10058000080087108E018F01080007118E018F016E
:10059000080007108E018F01080087128E018F015D
:1005A000080007128E018F01080087118E018F014C
:1005B00008000508103A850008000508203A850063
:1005C00008000508013A850008000508023A850080
:1005D00008000708023A870008000708043A870065
:1005E00008000708013A870008000708203A87003A
:1005F00008000708103A870008000708083A870033
:1006000008003D180516BD1885163D190514BD19BD
:1006100085143D1A8714BD1A07153D1B0714BD1B11
:10062000871642180716C218871508003C1D0800D7
:1006300050084002031D212B51080F02031C212BDF
:10064000051252084002031D2A2B53080F02031CF7
:100650002A2B851254084002031D332B55080F0224
:10066000031C332B051056084002031D3C2B570872
:100670000F02031C3C2B851058084002031D452B1C
:1006800059080F02031C452B87105A084002031D0E
:100690004E2B5B080F02031C4E2B07115C08400217
:1006A000031D572B5D080F02031C572B07105E0814
:1006B0004002031D602B5F080F02031C602B871292
:1006C0004C084002031D692B4D080F02031C692BC7
:1006D00007124E084002031D722B4F080F02031C25
:1006E000722B87110C1C08000C10C00A0800B60100
:1006F000B301B4013C1C7F2BBC01BC14862BBC1C79
:10070000842BBC013C15862BBC013C143C08B60074
:1007100064008A2B8B2B8C2B8D2B8E2BB41B0516F8
:10072000B41F0512B30B882BB40B882B0310B60C27
:10073000B608031D882B0030BB003C08BA005522C8
:020740000800AF
:084000000900030002000600A4
:02400E00CC33B1
:10420000010003000300030003000200020002009B
:1042100002000000000000000000FF00FF00FF009F
:10422000000000000000000000000000000000008E
:104230000000C000C000C000C000FF00FF00FF0081
:104240000100C300F300CF00FF00C300F300CF0064
:10425000FF00C300F300CF00FF00FF00FF00FF00DE
:10426000FF00FF00FF00FF00FF00FF00FF00FF0056
:10427000FF00FF00FF00FF00FF00FF00FF00FF0046
:10428000FF00FF00FF00FF00FF00FF00FF00FF0036
:10429000FF00FF00FF00FF00FF00FF00FF00FF0026
:1042A000FF00FF00FF00FF00FF00FF00FF00FF0016
:1042B000FF00FF00FF00FF00FF00FF00FF00FF0006
:1042C000FF00FF00FF00FF00FF00FF00FF00FF00F6
:1042D000FF00FF00FF00FF00FF00FF00FF00FF00E6
:1042E000FF00FF00FF00FF00FF00FF00FF00FF00D6
:1042F000FF00FF00FF00FF00FF00FF00FF00AA001B
:00000001FF
